:1000000074C100008EC100008CC100008AC10000D4
:1000100088C1000086C1000084C1000082C10000C8
:1000200080C100007EC100007CC100007AC10000D8
:1000300078C1000076C1000074C1000072C10000E8
:1000400070C100006EC100006CC100006AC10000F8
:1000500068C1000066C1000064C1000062C1000008
:1000600060C100005EC10000E5F078010000020000
:100070000303301004000005000008070209000017
:100080000A00000C00000D00000F0000100000111D
:10009000070012000013000007010000C8001090C4
:1000A00016112702003200120D0000320013001258
:1000B000290A002B0D000032003000003104043208
:1000C00003003505043608083707043803033907E9
:1000D000073C04053D08086000276101006A000034
:1000E0008000008100008200008300008400008501
:1000F00000009010009200009303009510019700FB
:1001000000980000000000000000005F00000007F1
:10011000000700147F147F14242A7F2A1223130857
:10012000646236495522500005030000001C22413C
:10013000000041221C0014083E081408083E08086C
:100140000050300000080808080800606000002027
:10015000100804023E5149453E00427F4000426182
:100160005149462141454B311814127F102745450E
:1001700045393C4A49493001710905033649494925
:1001800036064949291E0036360000005636000062
:1001900008142241001414141414004122140802FB
:1001A00001510906324979413E7E1111117E7F4984
:1001B0004949363E414141227F4141221C7F494904
:1001C00049417F090909013E4149497A7F080808E8
:1001D0007F00417F41002040413F017F08142241C0
:1001E0007F404040407F020C027F7F0408107F3E2A
:1001F0004141413E7F090909063E4151215E7F0987
:10020000192946464949493101017F01013F4040D2
:10021000403F1F2040201F3F4038403F63140814D8
:100220006307087008076151494543007F41410059
:1002300002040810200041417F0004020102044032
:1002400040404040000102040020545454787F484C
:100250004444383844444420384444487F38545453
:100260005418087E09010218A4A4A47C7F08040481
:100270007800447D40004080887A007F1028440048
:1002800000417F40007C041804787C08040478381E
:1002900044444438FC2424241818242418FC7C08E2
:1002A0000404084854545420043F4440203C404037
:1002B000207C1C2040201C3C4030403C442810281E
:1002C000441CA0A0A07C4464544C44000836410067
:1002D00000007F0000004136080010080810087870
:1002E00046414678FFFFFFFFFF0011241FBECFEFFE
:1002F000D8E0DEBFCDBF13E0A0E0B1E0E0E0F5E183
:1003000002C005900D92A039B107D9F723E0A0E90A
:10031000B3E001C01D92A83BB207E1F7C4D30C942F
:100320007E0A6ECE84B1836084B98AB18C6F8AB93B
:1003300087B18F6187B988B18B6088B98FE39CE9F9
:100340000197F1F700C00000089544988FE59AEEF8
:100350000197F1F700C00000449A8FE59AEE0197EB
:10036000F1F700C0000008959BB19370282F2C7FF7
:10037000922B9BB995B19C7F8370892B85B941984D
:10038000419A0895CF93C82F4298439880E0ECDFBC
:100390008C2FEADF439ACF910895CF93C82F429ACA
:1003A0004398892FE1DF8C2FDFDF439ACF910895A7
:1003B0000F931F93CF93DF93B5DFC7DF2FEF8DEE42
:1003C00092E0215080409040E1F700C0000008E634
:1003D00010E0F80184913196C591D49181110BC040
:1003E000CE01009759F0EFE9FFE03197F1F700C037
:1003F00000000197F6CFC6DFCE01CFDF0D5F1F4FA4
:10040000F1E004301F0729F72FEF81EE94E021502F
:1004100080409040E1F700C00000DF91CF911F9134
:100420000F91089587E0AEDF83E391E0B6CF882394
:1004300019F0813059F0089580E6A4DF80E097EA52
:10044000ACDF81E09FDF80E091E009C080E69ADFC9
:1004500080E097E2A2DF81E095DF80E090E09DCF31
:10046000A0E0B0E0E5E3F2E03BC48C01EB016A01FF
:10047000790180E587DFC80190DF81E583DFC60170
:100480008CDF82E57FDFCE0188DF83E57BDFC7017C
:1004900084DF80E277DFC80180DF81E273DFCE0195
:1004A0007CDF82E26FDFCDB7DEB7E8E035C4CF9204
:1004B000DF92EF92FF92CF93DF93EC012091000146
:1004C0003091010121503109409102015091030105
:1004D0004150510960E070E080E090E0C1DFC12C44
:1004E0008CE2D82EEE24E394F12CCE0156DF81E08D
:1004F000C81AD108E108F108C1F7DF91CF91FF9048
:10050000EF90DF90CF900895CF92DF92EF92FF921D
:100510000F931F93DA01A81BB90B1196F901E61B83
:10052000F70B3196AE9F6001AF9FD00CBE9FD00CF1
:100530001124E12CF12C94DFC114D104E104F10465
:1005400041F0C8012ADF81E0C81AD108E108F108AA
:10055000F3CF1F910F91FF90EF90DF90CF90089510
:10056000CF93DF93EA019B01AC017ADFCE0115DF67
:10057000DF91CF9108950F931F9389019A01AC01E8
:10058000C3DF1F910F9108950F931F93FB01BA01D1
:1005900089019A01AF01B8DF1F910F9108954F9221
:1005A0005F926F927F928F929F92AF92BF92CF9203
:1005B000DF92EF920F931F93CF93DF933C014B0198
:1005C000EA012901013019F486019EDF12C096016B
:1005D000A201D1DF9601A201B401CE01CCDF9601C8
:1005E000A401BE01C301D0DF9601A201BE01C30177
:1005F000CBDFEE2081F0A501B401C301B1DFA5017D
:10060000B201C301ADDFA501B401CE01A9DFA5018F
:10061000B201CE01A5DFDF91CF911F910F91EF9035
:10062000DF90CF90BF90AF909F908F907F906F9012
:100630005F904F900895AAE0B0E0E0E2F3E046C397
:100640002C017C836B833A01FA86E9861501882D9B
:100650004A01820E931E9201200F311F3A83298393
:10066000813049F5C40101979E838D839A012F5FE4
:100670003F4F38872F83E12C01E09C0149815A814B
:100680006F817885C20101968ADF4B815C81415080
:10069000510965012D813E816F81788589819A811B
:1006A00001967DDFC984DA8400E094014B815C818E
:1006B000B301C2010FC0E12C01E0940149815A81CC
:1006C000B301C2016CDF650194014B815C81B30110
:1006D00089819A8164DF2A96E2E114C32F923F92C6
:1006E0004F925F927F928F929F92AF92BF92CF92E2
:1006F000DF92EF92FF920F931F93CF93DF93FC0152
:10070000542E4901411102C055245394852D90E087
:100710009C018E179F0708F4CF0143E0220F331F7F
:100720004A95E1F7AB0141505109240F351FAC0147
:1007300041505109E5E05E9E400D511D112490DEAF
:1007400085E0E89E70011124C12CD12CE0EAEE1A5C
:10075000F10822242394312C0C2C02C0220C331CCF
:100760000A94E2F7712CA12CB12CF701EA0DFB1DC4
:10077000EC5FFE4FC491D0E0C221D321412C2097E1
:1007800011F0C40101C0C80108DE43945410F7CF32
:100790008FEFA81AB80AE5E0AE16B10431F77394EA
:1007A0005710E1CF8FEFC81AD80AE8E0CE16D1046F
:1007B00081F6DF91CF911F910F91FF90EF90DF9025
:1007C000CF90BF90AF909F908F907F905F904F9011
:1007D0003F902F900895A0E0B0E0E0EFF3E077C203
:1007E0003C016B01342E5901480186E0489F2001ED
:1007F0001124E701E99084019501432DB601C3015D
:100800006DDF640C751C88818052803698F3CDB7FB
:10081000DEB7E1E178C2ACE0B0E0E0E1F4E05CC278
:1008200087E880937A0087B1807F87B988B18F602D
:1008300088B9912CC12C61E070E09C2D906490935C
:100840007C0020E030E004E2A02EB12CE5E2F0E0F4
:10085000D22E82E0281305C01AE2A12EB12CEBE2C1
:10086000F0E0AB01022E01C0440F0A94EAF7D50173
:100870009C91942B9C93042F00951081102310833E
:100880008FE99FE00197F1F700C0000010917A0016
:10089000106410937A0010917A0016FDFCCFE0905E
:1008A0007800F0907900D5015C91902F95239C936E
:1008B0009081492B4083B4E6EB16F10458F581E0B2
:1008C000891540F1492D50E08A01000F111FA1E068
:1008D000B0E0AC0FBD1F0A0F1B1FD801ED92FC92B8
:1008E000BBE0EB2EF12CEC0EFD1EE40EF51ED70145
:1008F000CC9289E090E08C0F9D1F480F591FDA01C0
:10090000DC92AF0142505109D80115965C934E9389
:10091000149793942F5F3F4F2830310509F098CFFB
:10092000C394B4E0CB1289CFFDDCAB80BC80C9801E
:10093000DA80BF92AF92DF92CF9281ED92E09F93E7
:100940008F9380E993E09F938F9319D350E9E52E1D
:1009500053E0F52E00E010E029E53EEC41E062EDC9
:1009600070E08AE090E037DF0FB6F894DEBF0FBE8C
:10097000CDBF92E0991286C0EE24E394F12CAC1422
:10098000BD0410F0E12CF12CEBE0F0E0EC0FFD1FCA
:10099000EE0DFF1D9080692D80910A0190910B0151
:1009A00097D5E9E0F0E0EC0FFD1FEE0DFF1D808014
:1009B000682D80910E0190910F018AD501E010E021
:1009C000AC14BD0410F400E010E0E9E0F0E0EC0F3E
:1009D000FD1FE00FF11FD0806D2D809106019091D9
:1009E000070176D5EBE0F0E0EC0FFD1FE00FF11F03
:1009F000C0806C2D809108019091090169D5EE0CA1
:100A0000FF1CE1E0F0E0EC0FFD1FEE0DFF1D648127
:100A1000758180910C0190910D016CD5000F111F13
:100A2000E1E0F0E0EC0FFD1FE00FF11F6481758144
:100A300080910401909105015DD51F92CF921F9284
:100A4000DF921F928F921F929F9280EE92E09F936F
:100A50008F9380E993E09F938F9391D230E9E32EB7
:100A600033E0F32E00E010E020EE37E041E06CEDE3
:100A700070E08AE090E0AFDE0FB6F894DEBF0FBE04
:100A8000CDBF0EC081E0E82E83E0F82E00E010E03C
:100A900020E038EF41E06CED70E08AE090E09BDE12
:100AA0002C96ECE035C14F925F926F927F928F92BD
:100AB000AF92BF92CF92DF92EF92FF920F931F936C
:100AC000CF93DF9375DC81E0B2DC80E090E0EFDC77
:100AD000A9DC0FE0E02E03E0F02E00E010E02FEFA5
:100AE0003FEF41E066E170E08AE090E074DE82E191
:100AF000682E81E0782E2301C0E0D0E00091100143
:100B000010911101C017D10798F5BE0180E090E067
:100B1000A8D16B017C01B80180E090E0A2D120E077
:100B200030E04BE553E409D19B01AC01C701B601AC
:100B300004D16BD188248394A9E5AA2EAEECBA2EF9
:100B4000BFE1CB2ED12C10EEE12EFF24FA948B01C5
:100B50002AE030E042E350E065EE70E08AE090E0A9
:100B60006ADDF20161912F01CE01B2D42196C6CF88
:100B7000F1E2EF2EF3E0FF2E00E010E02FEF3FEF69
:100B800041E06AE770E08AE090E025DEC0E0D0E076
:100B90000091100110911101C017D10708F05DC03C
:100BA000BE0180E090E05DD16B017C01B80180E086
:100BB00090E057D120E030E04BE553E4BED09B01FC
:100BC000AC01C701B601B9D020D18824839449E58E
:100BD000A42E4EECB42E5FE1C52ED12CE0EEEE2E0D
:100BE000FF24FA948B012AE030E046E950E065EEFC
:100BF00070E08AE090E01FDDCE0162D4F3019191B4
:100C00003F01891741F11F929F931F928F93DF93AA
:100C1000CF9385E393E09F938F9380E993E09F9335
:100C20008F93ADD130E9E32E33E0F32E00E010E0F6
:100C300020E038EF41E064EB70E08AE090E0CBDD4B
:100C4000EDB7FEB73A960FB6F894FEBF0FBEEDBFF4
:100C500081E090E02BC021969BCF8AE5E82E83E0CF
:100C6000F82E00E010E020EE37E041E064EB70E0A9
:100C70008AE090E0B0DD90E6E92E93E0F92E2FEFC8
:100C80003FEF41E068EC70E08AE090E0A4DDC3DD76
:100C900029E7E22E23E0F22E2FEF3FEF41E060EF55
:100CA00070E08AE090E097DD80E090E0DF91CF9106
:100CB0001F910F91FF90EF90DF90CF90BF90AF907A
:100CC0008F907F906F905F904F9008952F923F92FA
:100CD0004F925F926F927F928F929F92AF92BF924C
:100CE000CF92DF92EF92FF920F931F93CF93DF93F8
:100CF000CDB7DEB7CA1BDB0B0FB6F894DEBF0FBE55
:100D0000CDBF09942A88398848885F846E847D84A1
:100D10008C849B84AA84B984C884DF80EE80FD80A3
:100D20000C811B81AA81B981CE0FD11D0FB6F89419
:100D3000DEBF0FBECDBFED0108950CD0E6C0DED002
:100D400040F0D5D030F021F45F3F19F0C7C0511109
:100D500010C1CAC0EBD098F39923C9F35523B1F35E
:100D6000951B550BBB27AA2762177307840738F01A
:100D70009F5F5F4F220F331F441FAA1FA9F333D079
:100D80000E2E3AF0E0E830D091505040E695001C2D
:100D9000CAF729D0FE2F27D0660F771F881FBB1FE9
:100DA000261737074807AB07B0E809F0BB0B802DC3
:100DB000BF01FF2793585F4F2AF09E3F510568F00F
:100DC0008DC0D7C05F3FECF3983EDCF386957795F6
:100DD0006795B795F7959F5FC9F7880F911D969511
:100DE000879597F90895E1E0660F771F881FBB1F6D
:100DF000621773078407BA0720F0621B730B840B1A
:100E0000BA0BEE1F88F7E095089598D088F09F57A9
:100E100090F0B92F9927B751A0F0D1F0660F771F46
:100E2000881F991F1AF0BA95C9F712C0B13081F026
:100E30009FD0B1E008959CC0672F782F8827B85FB6
:100E400039F0B93FCCF3869577956795B395D9F787
:100E50003EF490958095709561957F4F8F4F9F4F91
:100E60000895E89409C097FB3EF49095809570959D
:100E700061957F4F8F4F9F4F9923A9F0F92F96E9E6
:100E8000BB279395F695879577956795B795F1115B
:100E9000F8CFFAF4BB0F11F460FF1BC06F5F7F4FF8
:100EA0008F4F9F4F16C0882311F096E911C077230A
:100EB00021F09EE8872F762F05C0662371F096E813
:100EC000862F70E060E02AF09A95660F771F881FE2
:100ED000DAF7880F9695879597F9089597F99F67A0
:100EE00080E870E060E008959FEF80EC08950024B2
:100EF0000A941616170618060906089500240A947F
:100F000012161306140605060895092E0394000C04
:100F100011F4882352F0BB0F40F4BF2B11F460FF93
:100F200004C06F5F7F4F8F4F9F4F089557FD9058BC
:100F3000440F551F59F05F3F71F04795880F97FB9D
:100F4000991F61F09F3F79F0879508951216130657
:100F50001406551FF2CF4695F1DF08C01616170686
:100F60001806991FF1CF86957105610508940895BB
:100F7000E894BB2766277727CB0197F90895AEE061
:100F8000B0E0E4ECF7E0B0CE0D891E8986E08C83FA
:100F90001A8309838FEF9FE79E838D83AE01475E9F
:100FA0005F4F6F89788DCE01019608D0EF81F8856B
:100FB000E00FF11F10822E96E4E0B2CEABE0B0E07D
:100FC000E3EEF7E083CE6C017B018A01FC0117821E
:100FD0001682838181FFBFC1CE0101963C01F601DB
:100FE0009381F70193FD859193FF81917F01882380
:100FF00009F4ADC1853239F493FD859193FF819158
:101000007F01853221F4B60190E0C0D1E8CF912C68
:10101000212C312CFFE1F315D8F08B3279F038F424
:10102000803279F08332A1F4232D20611DC08D32EE
:1010300061F0803369F4232D216016C0832D826016
:10104000382EE32DE4603E2E2AC0F32DF8601DC03B
:1010500037FC2DC020ED280F2A3040F08E32B9F435
:1010600036FC75C1232D2064322E19C036FE06C011
:101070008AE0989E200D1124922E11C0EAE02E9E47
:10108000200D1124222EF32DF0623F2E08C08C3645
:1010900021F4832D8068382E02C0883641F4F70190
:1010A00093FD859193FF81917F018111B3CF982F9B
:1010B0009F7D9554933028F40C5F1F4F9FE39983D5
:1010C0000DC0833631F0833771F0833509F055C098
:1010D00020C0F801808189830E5F1F4F882483948C
:1010E000912C530112C02801F2E04F0E511CF8015F
:1010F000A080B18036FE03C0692D70E002C06FEFA2
:101100007FEFC50138D14C018201F32DFF773F2ECF
:1011100015C0280122E0420E511CF801A080B180C8
:1011200036FE03C0692D70E002C06FEF7FEFC5018E
:1011300017D14C01F32DF0683F2E820133FC19C00A
:10114000822D90E088169906A0F4B60180E290E026
:101150001DD12A94F5CFF50137FC859137FE819199
:101160005F01B60190E012D121102A9421E0821A89
:1011700091088114910479F7E1C0843611F0893621
:1011800039F5F80137FE07C0608171818281938152
:101190000C5F1F4F08C060817181072E000C880B07
:1011A000990B0E5F1F4FF32DFF763F2E97FF09C05F
:1011B00090958095709561957F4F8F4F9F4FF06808
:1011C0003F2E2AE030E0A3011DD1882E861844C0AE
:1011D000853731F4232D2F7EB22E2AE030E025C052
:1011E000932D997FB92E8F36C1F018F4883579F098
:1011F000AEC0803719F0883721F0A9C0E92FE0612F
:10120000BE2EB4FE0DC0FB2DF460BF2E09C034FE0F
:101210000AC0292F2660B22E06C028E030E005C0A3
:1012200020E130E002C020E132E0F801B7FE07C063
:1012300060817181828193810C5F1F4F06C0608144
:10124000718180E090E00E5F1F4FA301DBD0882EFC
:101250008618FB2DFF773F2E36FE0DC0232D2E7FE7
:10126000A22E891458F434FE0BC032FC09C0832D21
:101270008E7EA82E05C0B82CA32C03C0B82C01C0AC
:10128000B92CA4FE0FC0FE01E80DF11D8081803352
:1012900021F49A2D997EA92E09C0A2FE06C0B3940E
:1012A000B39404C08A2D867809F0B394A3FC10C0CF
:1012B000A0FE06C0B21480F4280C922C9B180DC01E
:1012C000B21458F4B60180E290E060D0B394F8CF45
:1012D000B21418F42B1802C0982C212CA4FE0FC0B5
:1012E000B60180E390E052D0A2FE16C0A1FC03C07C
:1012F00088E790E002C088E590E0B6010CC08A2D36
:10130000867851F0A1FE02C08BE201C080E2A7FC0A
:101310008DE2B60190E03AD0891430F4B60180E352
:1013200090E034D09A94F8CF8A94F301E80DF11D3F
:101330008081B60190E02AD08110F6CF222009F4F6
:101340004ECEB60180E290E021D02A94F7CFF6018C
:101350008681978102C08FEF9FEF2B96E2E1D2CC7E
:10136000FC010590615070400110D8F78095909570
:101370008E0F9F1F0895FC01615070400190011075
:10138000D8F7809590958E0F9F1F08950F931F9308
:10139000CF93DF93FB01238121FD03C08FEF9FEFEC
:1013A0002CC022FF16C04681578124813581421707
:1013B000530744F4A081B1819D012F5F3F4F3183DA
:1013C00020838C93268137812F5F3F4F378326837D
:1013D00014C08B01EC01FB010084F185E02D09951F
:1013E000892BE1F6D80116968D919C91179701965D
:1013F00017969C938E931697CE01DF91CF911F91F4
:101400000F910895FA01AA27283051F1203181F176
:10141000E8946F936E7F6E5F7F4F8F4F9F4FAF4FFC
:10142000B1E03ED0B4E03CD0670F781F891F9A1F0F
:10143000A11D680F791F8A1F911DA11D6A0F711DC3
:10144000811D911DA11D20D009F468943F912AE0CF
:10145000269F11243019305D3193DEF6CF010895B7
:10146000462F4770405D4193B3E00FD0C9F7F6CFE8
:10147000462F4F70405D4A3318F0495D31FD4052B0
:10148000419302D0A9F7EACFB4E0A6959795879546
:1014900077956795BA95C9F7009761057105089525
:1014A0009B01AC010A2E06945795479537952795D1
:1014B000BA95C9F7620F731F841F951FA01D089569
:1014C000F999FECF92BD81BDF89A992780B508950C
:1014D000262FF999FECF92BD81BDF89A019700B4ED
:1014E000021639F01FBA20BD0FB6F894FA9AF99A8D
:1014F0000FBE08950196272FECDFEACFF894FFCFB7
:101500004001F000B001B201AF01B601B301B50175
:10151000BF012801001200000080006801002801BE
:10152000001A0004008000080200280100120004D4
:10153000010080CE02002801001201040100809EFB
:1015400005005001001201040100803E0B00500113
:10155000002401040100807E1600500100480104AF
:10156000010080FE2C0001010000000401000000C9
:1015700000000653445249564520204154520072FF
:10158000035D07FF07A9008D04038D44028547A969
:10159000078D0503A9708D0A03A9018D0B03850929
:1015A000607D8A482053E488D0FA68AA8C8E07AD03
:1015B0007D07EE8E0760A9938DE202A9078DE302F5
:1015C000A20220DA07954320DA0795443543C9FF84
:1015D000F0F0CACA10EC3006E645D002E64620DA42
:1015E00007A2018144B545D543D0EDCA10F720D2FA
:1015F000074C9407A9038D0FD26CE202AD8E07CD84
:101600007F07D0ABEE0A03D003EE0B03AD7D070DD1
:101610007E07D08E20D207A900C547F0616CE0029A
:101620000720DA078DE00220DA078DE1022DE002C3
:10163000C9FFD0048547F0E9A900C547D03AADE01D
:10164000028580ADE10218EEFE076DFE078581A2DE
:101650000220DA07958020DA076DFE07E89580E81A
:10166000E00ED0EDA5828D0A07A5838D0B07A58D11
:101670006DFE078D0D07A90A8D8E074C9407A2FFFA
:101680009AA90A85C9A90085098DF803A9FD8D01CC
:10169000D3A9A948A97948A9B748A95448A56A1067
:1016A00002A9A0856A4C94EFFFFFFFFFFFFFFFFF39
:1016B000FFFFFFFFFFFFFFFFFFFFFFFFFFFFFFFF3A
:1016C000F3FFFFFFFFFFFFFFFFFFFFFFFFFFFFFF36
:1016D000FF56616C7565733A2025692C20256900D9
:1016E00058503A204125692C20584D3A2025692C24
:1016F0002059503A2025692C20594D3A204125691E
:10170000004E6F74206465746563746564210057CE
:10171000726974696E6720454550524F4D2E2E2ECA
:1017200000566572696679696E6720454550524F6B
:101730004D2E2E2E00566572696679206572726F85
:1017400072206174203078253033783A2025303289
:101750007820213D202530327800446F6E652100CD
:10176000446574656374696E6720746F756368732C
:10177000637265656E2E2E2E004E6F7720666C614B
:101780007368205344726976652E6865782100007D
:00000001FF
